:0400000080316928BA
:1000080080310310003003180130F10021009111F4
:100018002400951F10281128122895132000921DDE
:1000280016281728182892112400151F1C281D2887
:1000380024281108F0007008F1001513151624285B
:100048002000911D2828292866282400941D2D2881
:100058002E286428141D312832284828941A352857
:10006800362842281108F0007008F100780891003D
:100078000310003003180130F8004528FF309100C4
:10008800452815166400642814194B284C28642840
:10009800141C4F2850286428941A53285428592887
:1000A8001108F0007008F1005F281108F0007008CE
:1000B8002000AB005F2824001516642864286428F3
:1000C8002000911121009115090088018131E5294D
:1000D8000034233430342A3439343834373436341D
:1000E80035343434333432343134031000300318A7
:1000F80001302000AA000310003003180130A900C5
:100108000030A3000030A2000030A1000030A000A1
:100118000030A8000030A7000030A6000030A5007D
:100128007F30F6007608210095058B0198308E0007
:10013800073020008E000F3021008D0020008D1622
:1001480024000D148D140D158D15F030F600760869
:1001580023008D057E30210099000F3098008131F1
:10016800DC2180311330210097008B170B17911574
:1001780020009111D028D028031000300318013036
:10018800AB008D12D8280310003003180130AB00E3
:100198008D16D828D828D8282B08113A0319C02832
:1001A800333A0319C728D8282408031DDC282B292B
:1001B8000130F6002A0AE128F635890BE02876088E
:1001C800FF3AF70077088E050130F600290AED2876
:1001D800F635890BEC2876080D050319F428F5285F
:1001E8001F2900302302031D032900302202031DAA
:1001F800032901302102031D0329F4302002031CC6
:100208000629072915290030A8000030A70000306A
:10021800A6000030A5000310003003180130A40028
:100228001F290130A0070030A13D0030A23D003059
:10023800A33D1F291F290130F6002A0A2429F63573
:10024800890B23297608F70077088E04D028013017
:10025800F6002A0A3029F635890B2F297608FF3A45
:10026800F70077088E050130F600290A3C29F63593
:10027800890B3B2976080D05031D432944297D294F
:1002880000302802031D522900302702031D52297D
:1002980000302602031D5229C8302502031C5529A7
:1002A800562973290030A3000030A2000030A100B5
:1002B8000030A000A4010314A40D0330F600760852
:1002C800F20029088131BF2180316D3E20002A07C4
:1002D80080310A008131F7007708F800862901305B
:1002E800A5070030A63D0030A73D0030A83D86296F
:1002F80086290030A8000030A7000030A600003092
:10030800A50086290130F6002A0A8B29F635890BC3
:100318008A297608F70077088E0428082704260417
:100328002504031D98299929D0280130F60076085C
:10033800A90704302902031CA229A329D0280310E5
:10034800003003180130A9000130F6007608AA072A
:1003580003302A02031CB129B229D0280310003027
:1003680003180130AA00D028D028D028D028D028B7
:10037800D02880316928F5000310003003180130B7
:10038800F400C629751CC929CA29CF297208F300A7
:100398007308F407CF290310F20D0310F50CF508C4
:1003A800031DD729D829C629D9297408DB290800AB
:1003B8002E3024009500E430920016109710171084
:1003C80008008131EC218131F80020008031792842
:0203D800BB3434
:00000001FF
